:020000000A28CC
:10000800FF000308FB000A08FC00352C3C30840084
:1000180070300F20172864008001840A0406031931
:10002800003404061028F030831685008601073056
:1000380083129F0042308316810083129010901122
:100048001012901210148B010030A2270038031DE3
:100058004D280130A2278312BC000230A227831248
:10006800DE000330A2278312DF000430A2278312A8
:10007800E7000530A2278312D9000630A227831291
:10008800EA000730A2278312EC000830A227831267
:100098005D2819308312BC000630DE000430DF0012
:1000A800E701E70A1E30D9001630EA000630EC00F6
:1000B8000F30C0006708E60083160C1483128B16F5
:1000C8000B178B176E17EE1FA528EE1305305A0273
:1000D80003187028AC277628DD08031D75280B2126
:1000E8007628C7216F1E7E286608063A03198028DD
:1000F8003F087F284008D400C326EF1F6F1B8628BF
:10010800EF1EA2286D14C401DD0146080A3A47040F
:1001180003197B22013047022D3003194602031CC4
:100128009E2847304202031C9C287B22C201A52836
:10013800C20AA528C60A0319C70AA528C601C70105
:100148006E106E1F67286E13092505305A02031CAE
:10015800DA0A6F1EFA280530F000F0080319B928EA
:10016800C3236F18B928F003B128962783126A08A9
:1001780065020318C3286C0865020318C6284008DE
:10018800BF00C728BF01EB08031DFC28C3080319DB
:10019800CF28C303FC28DF08031DD428EF11DB2870
:1001A800DE08031DD928EF15DB280830EF06EF1D00
:1001B800DF285F08E0285E08C30067080E3A031DC1
:1001C800EC280D3066020318EB28E60AEC28E60155
:1001D80067080F3A03190C27E6080319FC28DD0104
:1001E800DD0ADC01BE01BE03C101FC285E08C300B4
:1001F8006D1C67280A30440203180429C40A6728BA
:10020800EE1E0729612483126D10EB016728EE1199
:100218006F1D6F1B1129EF1E1329EF101429EF14FE
:10022800EB08031D23296F1F1C29EE1523272329FB
:10023800EF1EEF192229EE1523272329F0226B0B35
:100248002C29EE152327EF1C2C290B30E000E900A0
:100258006B08023A031D3729EE152327EF1C3729AF
:100268000B30E300E1006B08033A031D44295B08E7
:100278007A276808E9006208E0000B30E300E10033
:100288006B08043A031D58291930E3000B30E100CC
:1002980019303C023C08031C5429E73E4A275829D8
:1002A800193C4A270A30E1006B08053A031D622908
:1002B8005E084A270F30E3001930E1006B08063A60
:1002C800031D6B295F084A270F30E300E1006B0824
:1002D800073A031D90290B30E90067080E3A031D01
:1002E800772910307C2967080F3A031D7E290E30C4
:1002F800E000872967087A276208E000E808031900
:1003080087296808E900EF1C8C290B30E000E90018
:100318001530E3001330E1006B08083A031D9A29F1
:1003280059084A270B30E1001730E3006B08093AF7
:10033800031DA4296A084A271230E3000B30E100A4
:100348006B080A3A031DAE296C084A271430E300EB
:100358000B30E1006B080B3A031DB82940084A2707
:100368002330E3000B30E10063087F23CE006108EF
:100378007F23CD00EE19CD1769087F23CC006008D4
:100388007F23CB000800C1080319CC29C10308004A
:100398005908C100522A5D0BD229EC2D512E5D0B54
:1003A800D629A8265D08023A03193225080001302B
:1003B80058020318E129D80A0800D8015D0BE5297D
:1003C8005B275D08023A03195A2508005D0BED29E1
:1003D800EC2D0E2E5D0BF129B6245D08023A0319A7
:1003E800322508005D0B012A163054020318FE2935
:1003F800D40A012A0B210230DD005D08023A031DF0
:10040800080054083F0203180B2AD4030800DD0132
:100418000800013058020318132AD80A0800D80126
:100428005D0B172A38275D08023A03198C24080047
:100438005D0B1F2AA52D0E2E5D0B232AA8265D080D
:10044800023A0319E02408005D0B2B2AA52D512E32
:10045800013058020318322AD80A0800D8015D0B67
:10046800362A5B275D08023A03198C2408005D0BC5
:100478003E2AB6245D08023A0319E0240800013038
:1004880058020318492AD80A0800D8015D0B4D2ADA
:1004980038275D08023A03195A2508006608013A08
:1004A8000319CF29033A0319D329013A0319DB2980
:1004B800073A0319EA29013A0319EE29033A0319FD
:1004C800F629013A03190D2A0F3A03191C2A013A91
:1004D8000319202A033A0319282A013A03192C2A56
:1004E800073A03193B2A013A031D0800432AEF1B68
:1004F8006E18882A6F1E882A6E140B306B02031838
:10050800872AEB0A882AEB016B0B8F2A3B30F10014
:100518006408F526E4006B08023A031D982A173090
:10052800F1006508F526E5006B08033A031DA12ACA
:100538006F1BA02AEF1EA12ADB016B08043A031DDA
:10054800AA2A3230F1003C08F526BC006B08053AAF
:10055800031DB32A6330F1005E08F526DE006B0840
:10056800063A031DBC2A6330F1005F08F526DF0058
:100578006B08073A031DCB2A0F30F1006708F526F0
:10058800E7006F1BC92AEF1ECB2A6708E6006B0835
:10059800083A031DD42A6330F1005908F526D9001A
:1005A8006B08093A031DDD2A1730F1006A08F526A1
:1005B800EA006B080A3A031DE62A1730F1006C08B6
:1005C800F526EC006B080B3A031D08001230F10009
:1005D8004008F526C0000800EE154A08F40049084E
:1005E800F300E301E101E9016F1C342B03307402CD
:1005F800E83003197302031C092B342B9C30F307D2
:100608000318F40AFF30F407E30A00307402643078
:1006180003197302031C182B022BF630F307031877
:10062800F40AFF30F407E10A003074020A300319B3
:1006380073020318112B7308E900E308EE1C2D2B35
:1006480003192B2B6108E9006308E100EE110A3059
:10065800302B031D312B0B30E3001D30E000080068
:100668000A30E000E900E100E3000800003052022F
:10067800031D482B00305102031D482B083050023F
:10068800031D482B00304F02031C5F2B0030CF079F
:10069800F83003110318013E031DD007FF30031182
:1006A8000318013E031DD107FF3003110318013E53
:1006B800031DD207752B4030CF073A3003110318BA
:1006C800013E031DD0070F3003110318013E031D1F
:1006D800D107003003110318013E031DD2076E171E
:1006E800BD01F3303D0203187B2BBD0A0800BD0194
:1006F8000430EF060800F300003A03193F34013ACA
:1007080003190634033A03195B34013A03194F34C9
:10071800073A03196634013A03196D34033A031989
:100728007D34013A031907340F3A03197F34013A2B
:1007380003196F34033A03194034043A0319503447
:10074800013A031978341F3A03197734023A031926
:100758005434013A03197134073A03195E34013AE3
:1007680003197934023A031973340E3A03195834C9
:10077800043A031963343E3A03197C340034802563
:100788006F1C0800CC30C925BE30C925302683121D
:1007980003134808D3003026831203134808D500F2
:1007A800D51FE42BD308031DDD2B5509013ED500C9
:1007B800DF2BFF30D5065309023ED300EE14E52B9C
:1007C800EE105508CA005308C9000A30F700F801AE
:1007D8004A08F6004908F500DC2604300310F60C38
:1007E800F50CFF3E031DF22B7508C9007608CA00F8
:1007F80008008601F03085056F12851A6F166F1E86
:10080800332C0514EF17851AEF13051085146F178D
:10081800851A6F1385100515EF16851AEF120F301C
:100828008504C508031D1B2C4E0886000510450BC2
:10083800202C4D08860085104508023A031D272CF8
:100848004C08860005114508033A031D312C4B0856
:10085800831386008511C5010800C50A0800EB014D
:100868000800831203130B1D4E2C0A305402031C7C
:10087800412C13305402031C422C6E16EE173A23F7
:1008880013305402031CFD2357088E0056088F00AE
:100898000B110C100C1C5A2C0A305402031C552C3A
:1008A8006E166F1E592C0F3085040C107C088A00B8
:1008B8007B088300FF0E7F0E0900F10100308D26B2
:1008C80083123C08F10001308D2683125E08F10086
:1008D80002308D2683125F08F10003308D268312C3
:1008E8006708F10004308D2683125908F10005309D
:1008F8008D2683126A08F10006308D2683126C0853
:10090800F10007308D2683124008F10008308D2E43
:100918000B2103305C02031CA82CB42C4B08831356
:10092800CE00CC01CD01A62C4C08CE004B08831379
:10093800CD00CC01A62C4D08CE004C08CD004B08AC
:100948008313CC00CB01B22C5C08003A0319922C1B
:10095800013A0319982C033A03199F2CDC0A080062
:10096800DD010800C92C7F30BE2C7730BE2C6330E7
:10097800BE2C2330F100DC2CF101F10ADC2CF10152
:100988000230DD000430DC00DC2C5C08003A03197E
:10099800B72C013A0319B92C033A0319BB2C013AB5
:1009A8000319BD2C073A0319C02C013A0319C32CAB
:1009B80071088827DC0A08000B21F22C7F30F1002F
:1009C800DD01052D7730EB2C6330EB2C2330F10063
:1009D800052DF101F10A052DF101052D5C08003AFC
:1009E8000319E22C013A0319E62C033A0319E82CFF
:1009F800013A0319EA2C073A0319ED2C013A0319B5
:100A0800F02C71088827DC0308003B305B020318D0
:100A18000F2DDB0A1E2DDB013B3064020318162D57
:100A2800E40A1E2DE4011730650203181D2DE50A9E
:100A38001E2DE5015B081E3A031D2E2DE408031D3B
:100A48002E2DE50803196E1D2E2D3C085B07E73E89
:100A5800DB006E11640B08006E1508000B21432D96
:100A6800FE30F100DD01562DDC303F2D9C303F2D4E
:100A780088303F2D8030F100562DF101562D5C084D
:100A8800003A0319342D013A0319382D033A031992
:100A98003A2D013A03193C2D073A03193E2D013A24
:100AA8000319412D71088827DC0308000B21033046
:100AB8005C02031C722D7E2D4E08CB00CC01682DE4
:100AC8004D08CB004E08CC00CD01702D4C08CB0052
:100AD8004D08CC004E08CD00CE017C2D5C08003AB4
:100AE8000319602D013A0319642D033A03196A2D7D
:100AF800DC0A0800DD0108006E126E1E812DB52784
:100B08005330F100F10B862D5330F200F20B8A2D91
:100B18008316031305162130F300F30B912D83126E
:100B280003136F10051A08004330F400F40B9A2DD4
:100B38004330F500F50B9E2D83120313051A6F142D
:100B4800080007305C020318C52D0130F2005C086C
:100B5800073C013EB12D0310F20DFF3E031DAF2DE2
:100B68007208FF3ABE05DC0AF10171084B3E8400A9
:100B780083133E088005F10A043071020318080047
:100B8800B92D0230DD00DC010800F10083126E127D
:100B98006E1ECC2DF201B5270000711CD72D8312D3
:100BA80003130516DA2D8312031305121330F3000D
:100BB800F30BDC2D8316031305160000000000005C
:100BC8000310F10CF20A0830720203180800CF2D46
:100BD80007305C0203180A2E0130F2005C0AF62D79
:100BE8000310F20DFF3E031DF42D7208FF3ABE05F7
:100BF800DC0AF10171084B3E840083133E0880052E
:100C0800F10A0430710203180800FE2D0230DD00DD
:100C1800DC0108000B2107305C0203182E2E01307E
:100C2800F2005C08073C013E1B2E0310F20DFF3E4C
:100C3800031D192E7208BE04DC0AF10171084B3E2F
:100C4800840083133E088005F10A043071020318FA
:100C58000800222EDD01080083126E126E1E322E4D
:100C6800F101B527F201F20AF20B382E83160313AD
:100C78000516F301F30AF30B3F2E83120313031037
:100C8800C80C051AC8171530F400F40B492EF10AE0
:100C98000830710203180800352E0B2107305C025A
:100CA80003186F2E0130F2005C0A5C2E0310F20D5F
:100CB800FF3E031D5A2E7208BE04DC0AF1017108BA
:100CC8004B3E840083133E088005F10A043071020C
:100CD80003180800632EDD010800F4000830F50051
:100CE800F6017408F70007300310F70CFF3E0310F5
:100CF800031D792E760D7704F6000310F40D7308A2
:100D08007602031C892E7308F602F50B752E7608F9
:100D18000800F20083169C188E2E72089B0071083A
:100D28009A009C13031083128B1B03148B138316D6
:100D38001C1555309D00AA309D009C141C11031CE5
:100D4800080083128B170800AE2E0230DD00043035
:100D5800DC00C12E5C08003A0319C12E013A0319C0
:100D6800C12E033A0319C12E013A0319C12E073ABD
:100D78000319C12E013A0319A92EDC0A08006430B0
:100D8800F700F8015408F500F601DC267508A23EC4
:100D9800F10076080318013EF83EF200D600003054
:100DA800F50056086C27F30071087307D700080090
:100DB800F901FA01751CE62E7708F9070318FA0AF3
:100DC8007808FA070310F70DF80D0310F60CF50C68
:100DD80076087504031DDE2E7A08F6007908F500FA
:100DE8000800F2006F1F002F710872020318FE2E10
:100DF800F20AFF2EF201EE16EF1E0A2FF20803196F
:100E0800072FF203092F7108F200EE167208080086
:100E18006608F10053085B0766076407E6000D30B3
:100E2800F30066087126E6007106031D08000D3000
:100E380066020318212FE60A0800E6010800650883
:100E48007A27E808031D2A2F0B302B2F6808E300A8
:100E58006208E10064087A276808E9006208E0008F
:100E6800EE156F19EE11080003305C020318462FC7
:100E7800DC0A4D08CE004C08CD004B088313CC008B
:100E8800CB0108000230DD00DC010800F3007A27FE
:100E98006808E9006208E000E908031D552F0B30D7
:100EA800E900EF1C08000B30E000E90008000330FF
:100EB8005C020318682FDC0A4C08CB004D08CC00F4
:100EC8004E08CD00CE0108000230DD00DC0108002C
:100ED800F600F70175087618F7070310F50D0310EB
:100EE800F60CF608031D6E2F77080800F400E801D9
:100EF800E201812FF630F407E80A0A307402031879
:100F08007E2F7408E2000800F200F30173084B3EDC
:100F18008400831372088005F30A043073020318EF
:100F280008008A2F80256F1C0800CC30C925443062
:100F3800C92583120516831605160800F1008316C5
:100F48009C18A32F71089B009C131C141A080800F6
:100F58006D30CE005C30CD001030CC005030CB006E
:0E0F68000800831203130512831605120800F9
:02400E000A3F67
:00000001FF
